******************************************************************************
             TMS320C2000 Linker PC v18.12.7                    
******************************************************************************
>> Linked Tue Nov 17 17:27:52 2020

OUTPUT FILE NAME:   <usb_ex4_dev_bulk_my.out>
ENTRY POINT SYMBOL: "code_start"  address: 00080000


MEMORY CONFIGURATION

         name            origin    length      used     unused   attr    fill
----------------------  --------  ---------  --------  --------  ----  --------
PAGE 0:
  RAMM0                 00000123   000002dd  00000000  000002dd  RWIX
  RAMLS0                00008000   00000800  0000012f  000006d1  RWIX
  RAMLS1                00008800   00000800  00000000  00000800  RWIX
  RAMLS2                00009000   00000800  00000000  00000800  RWIX
  RAMLS3                00009800   00000800  00000000  00000800  RWIX
  RAMLS4                0000a000   00000800  00000000  00000800  RWIX
  RAMD0                 0000b000   00000800  00000000  00000800  RWIX
  RAMGS14               0001a000   00001000  00000000  00001000  RWIX
  RAMGS15               0001b000   00000ff8  00000000  00000ff8  RWIX
  BEGIN                 00080000   00000002  00000002  00000000  RWIX
  FLASHA                00080002   00001ffe  00000000  00001ffe  RWIX
  FLASHB                00082000   00002000  00002000  00000000  RWIX
  FLASHC                00084000   00002000  0000158e  00000a72  RWIX
  FLASHD                00086000   00002000  0000012f  00001ed1  RWIX
  FLASHE                00088000   00008000  00000111  00007eef  RWIX
  FLASHF                00090000   00008000  00000a14  000075ec  RWIX
  FLASHG                00098000   00008000  00000000  00008000  RWIX
  FLASHH                000a0000   00008000  00000000  00008000  RWIX
  FLASHI                000a8000   00008000  00000000  00008000  RWIX
  FLASHJ                000b0000   00008000  00000000  00008000  RWIX
  FLASHK                000b8000   00002000  00000000  00002000  RWIX
  FLASHL                000ba000   00002000  00000000  00002000  RWIX
  FLASHM                000bc000   00002000  00000000  00002000  RWIX
  FLASHN                000be000   00001ff0  00000000  00001ff0  RWIX
  RESET                 003fffc0   00000002  00000000  00000002  RWIX

PAGE 1:
  BOOT_RSVD             00000002   00000121  00000000  00000121  RWIX
  RAMM1                 00000400   000003f8  000003f8  00000000  RWIX
  RAMLS5                0000a800   00000800  000007b0  00000050  RWIX
  RAMD1                 0000b800   00000800  00000000  00000800  RWIX
  RAMGS0                0000c000   00001000  00000000  00001000  RWIX
  RAMGS1                0000d000   00001000  00000000  00001000  RWIX
  RAMGS2                0000e000   00001000  00000000  00001000  RWIX
  RAMGS3                0000f000   00001000  00000000  00001000  RWIX
  RAMGS4                00010000   00001000  00000000  00001000  RWIX
  RAMGS5                00011000   00001000  00000000  00001000  RWIX
  RAMGS6                00012000   00001000  00000000  00001000  RWIX
  RAMGS7                00013000   00001000  00000000  00001000  RWIX
  RAMGS8                00014000   00001000  00000000  00001000  RWIX
  RAMGS9                00015000   00001000  00000000  00001000  RWIX
  RAMGS10               00016000   00001000  00000000  00001000  RWIX
  RAMGS11               00017000   00001000  00000000  00001000  RWIX
  RAMGS12               00018000   00001000  00000000  00001000  RWIX
  RAMGS13               00019000   00001000  00000000  00001000  RWIX
  CPU2TOCPU1RAM         0003f800   00000400  00000000  00000400  RWIX
  CPU1TOCPU2RAM         0003fc00   00000400  00000000  00000400  RWIX


SECTION ALLOCATION MAP

 output                                  attributes/
section   page    origin      length       input sections
--------  ----  ----------  ----------   ----------------
codestart 
*          0    00080000    00000002     
                  00080000    00000002     F2837xD_CodeStartBranch.obj (codestart)

.cinit     0    00088000    00000111     
                  00088000    00000046     usblib_coff.lib : usbhostenum.obj (.cinit)
                  00088046    00000039     usb_ex4_dev_bulk_structs.obj (.cinit)
                  0008807f    00000018     usb_ex4_dev_bulk.obj (.cinit)
                  00088097    00000015     usblib_coff.lib : usbdbulk.obj (.cinit:_g_pui8BulkDeviceDescriptor)
                  000880ac    0000000f     device.obj (.cinit)
                  000880bb    0000000e     rts2800_fpu32.lib : exit.c.obj (.cinit)
                  000880c9    0000000e     usblib_coff.lib : usbtick.obj (.cinit)
                  000880d7    0000000d                     : usbmode.obj (.cinit)
                  000880e4    0000000c                     : usbdbulk.obj (.cinit:_g_pui8BulkDescriptor)
                  000880f0    00000007                     : usbdbulk.obj (.cinit:_g_psBulkSections)
                  000880f7    00000005     rts2800_fpu32.lib : _lock.c.obj (.cinit:__lock)
                  000880fc    00000005                       : _lock.c.obj (.cinit:__unlock)
                  00088101    00000005     scistdio.obj (.cinit)
                  00088106    00000005     usblib_coff.lib : usbdenum.obj (.cinit)
                  0008810b    00000004     ustdlib.obj (.cinit)
                  0008810f    00000002     --HOLE-- [fill = 0]

.stack     1    00000400    000003f8     UNINITIALIZED
                  00000400    000003f8     --HOLE--

.reset     0    003fffc0    00000002     DSECT
                  003fffc0    00000002     rts2800_fpu32.lib : boot28.asm.obj (.reset)

.pinit     0    00082000    00000000     UNINITIALIZED

.TI.ramfunc 
*          0    00086000    0000012f     RUN ADDR = 00008000
                  00086000    00000043     driverlib_coff.lib : flash.obj (.TI.ramfunc:_Flash_initModule)
                  00086043    0000002d                        : flash.obj (.TI.ramfunc:_Flash_setBankPowerMode)
                  00086070    00000026                        : flash.obj (.TI.ramfunc:_Flash_setWaitstates)
                  00086096    0000001e                        : flash.obj (.TI.ramfunc:_Flash_setPumpPowerMode)
                  000860b4    00000018                        : flash.obj (.TI.ramfunc:_Flash_disableCache)
                  000860cc    00000018                        : flash.obj (.TI.ramfunc:_Flash_disablePrefetch)
                  000860e4    00000018                        : flash.obj (.TI.ramfunc:_Flash_enableCache)
                  000860fc    00000018                        : flash.obj (.TI.ramfunc:_Flash_enablePrefetch)
                  00086114    00000017                        : flash.obj (.TI.ramfunc:_Flash_enableECC)
                  0008612b    00000004                        : sysctl.obj (.TI.ramfunc)

GETBUFFER 
*          0    0003f800    00000000     DSECT

GETWRITEIDX 
*          0    0003f800    00000000     DSECT

PUTREADIDX 
*          0    0003f800    00000000     DSECT

.text.1    0    00082000    00002000     
                  00082000    00000376     usblib_coff.lib : usbhostenum.obj (.text:_USBHostIntHandlerInternal)
                  00082376    00000261     scistdio.obj (.text)
                  000825d7    0000024e     device.obj (.text)
                  00082825    0000021f     driverlib_coff.lib : sysctl.obj (.text:_SysCtl_setClock)
                  00082a44    0000020d     usb_ex4_dev_bulk.obj (.text)
                  00082c51    000001ad     usblib_coff.lib : usbdconfig.obj (.text:_USBDeviceConfig)
                  00082dfe    00000127     driverlib_coff.lib : sysctl.obj (.text:_SysCtl_setAuxClock)
                  00082f25    00000127     usblib_coff.lib : usbdenum.obj (.text:_USBDGetDescriptor)
                  0008304c    000000de                     : usbdenum.obj (.text:_USBDEP0StateTxConfig)
                  0008312a    000000cd     usb_hal.obj (.text)
                  000831f7    000000ca     usblib_coff.lib : usbdenum.obj (.text:_USBDeviceEnumHandler)
                  000832c1    000000c4     usb_hal.obj (.text:retain)
                  00083385    000000ae     usblib_coff.lib : usbbuffer.obj (.text:_HandleRxAvailable)
                  00083433    000000ad                     : usbdenum.obj (.text:_USBDCDInit)
                  000834e0    0000009c     rts2800_fpu32.lib : fd_add28.asm.obj (.text)
                  0008357c    0000009b     usblib_coff.lib : usbdbulk.obj (.text:_USBDBulkCompositeInit)
                  00083617    0000009a                     : usbdenum.obj (.text:_USBDeviceIntHandlerInternal)
                  000836b1    00000095                     : usbdenum.obj (.text:_USBDSetInterface)
                  00083746    0000008b     rts2800_fpu32.lib : fd_div28.asm.obj (.text)
                  000837d1    0000008a     usblib_coff.lib : usbbuffer.obj (.text:_ScheduleNextTransmission)
                  0008385b    00000089     driverlib_coff.lib : usb.obj (.text:_USBDevEndpointConfigSet)
                  000838e4    00000088     usblib_coff.lib : usbdenum.obj (.text:_USBDClearFeature)
                  0008396c    00000088     rts2800_fpu32.lib : fs_div28.asm.obj (.text)
                  000839f4    00000085     driverlib_coff.lib : interrupt.obj (.text:_Interrupt_clearIFR)
                  00083a79    0000007f     usblib_coff.lib : usbmode.obj (.text:_USB0OTGModeIntHandler)
                  00083af8    00000071                     : usbdenum.obj (.text:_USBDSetConfiguration)
                  00083b69    0000006e     driverlib_coff.lib : usb.obj (.text:_USBDevEndpointStallClear)
                  00083bd7    0000006c     usblib_coff.lib : usbdenum.obj (.text:_USBDGetStatus)
                  00083c43    0000006b                     : usbdenum.obj (.text:_USBDSetFeature)
                  00083cae    0000006b     driverlib_coff.lib : usb.obj (.text:_USBEndpointDataGet)
                  00083d19    0000006a                        : usb.obj (.text:_USBDevEndpointStatusClear)
                  00083d83    00000069     usblib_coff.lib : usbdconfig.obj (.text:_USBDeviceConfigAlternate)
                  00083dec    00000068     driverlib_coff.lib : sysctl.obj (.text:_SysCtl_getDeviceParametric)
                  00083e54    00000066                        : usb.obj (.text:_USBFIFOConfigSet)
                  00083eba    00000066     usblib_coff.lib : usbdma.obj (.text:_USBLibDMAInit)
                  00083f20    0000005e     driverlib_coff.lib : sysctl.obj (.text:_SysCtl_selectOscSource)
                  00083f7e    0000005e     usblib_coff.lib : usbdbulk.obj (.text:_USBDBulkPacketRead)
                  00083fdc    00000024                     : usbdbulk.obj (.text:_HandleDisconnect)

.text.2    0    00084000    0000158e     
                  00084000    0000005c     usblib_coff.lib : usbdenum.obj (.text:_USBDEP0StateTx)
                  0008405c    0000005b                     : usbdbulk.obj (.text:_USBDBulkInit)
                  000840b7    0000005b     driverlib_coff.lib : usb.obj (.text:_USBDevEndpointStall)
                  00084112    00000059                        : usb.obj (.text:_USBEndpointDataSend)
                  0008416b    00000058     usblib_coff.lib : usbdenum.obj (.text:_USBDStringIndexFromRequest)
                  000841c3    00000057     driverlib_coff.lib : usb.obj (.text:_USBIntStatus)
                  0008421a    00000056     rts2800_fpu32.lib : boot28.asm.obj (.text)
                  00084270    00000054     driverlib_coff.lib : usb.obj (.text:_USBEndpointDataPut)
                  000842c4    00000053     usblib_coff.lib : usbringbuf.obj (.text:_USBRingBufWrite)
                  00084317    00000052     driverlib_coff.lib : gpio.obj (.text:_GPIO_setPadConfig)
                  00084369    00000051                        : sysctl.obj (.text:_SysCtl_getClock)
                  000843ba    0000004f                        : usb.obj (.text:_USBHostEndpointStatusClear)
                  00084409    0000004e     usblib_coff.lib : usbdbulk.obj (.text:_ProcessDataFromHost)
                  00084457    0000004e                     : usbdbulk.obj (.text:_USBDBulkPacketWrite)
                  000844a5    0000004e                     : usbdenum.obj (.text:_USBDGetInterface)
                  000844f3    0000004b     driverlib_coff.lib : interrupt.obj (.text:_Interrupt_disable)
                  0008453e    0000004a     usblib_coff.lib : usbdenum.obj (.text:_USBDReadAndDispatchRequest)
                  00084588    0000004a     driverlib_coff.lib : usb.obj (.text:_USBDevEndpointDataAck)
                  000845d2    00000048                        : usb.obj (.text:__USBIndexWrite)
                  0008461a    00000047                        : usb.obj (.text:_USBEndpointDataAvail)
                  00084661    00000044     usblib_coff.lib : usbdcdesc.obj (.text:_USBDCDConfigDescGet)
                  000846a5    00000043                     : usbbuffer.obj (.text:_USBBufferEventCallback)
                  000846e8    00000043     driverlib_coff.lib : usb.obj (.text:_USBHostEndpointDataAck)
                  0008472b    00000043     usblib_coff.lib : usbringbuf.obj (.text:_USBRingBufAdvanceWrite)
                  0008476e    0000003f     driverlib_coff.lib : usb.obj (.text:_USBEndpointStatus)
                  000847ad    0000003e                        : sci.obj (.text:_SCI_setConfig)
                  000847eb    0000003d                        : interrupt.obj (.text:_Interrupt_initModule)
                  00084828    0000003b     usblib_coff.lib : usbdconfig.obj (.text:_GetEPDescriptorType)
                  00084863    0000003b                     : usbdenum.obj (.text:_USBDGetConfiguration)
                  0008489e    0000003b     driverlib_coff.lib : usb.obj (.text:_USBIntEnableControl)
                  000848d9    0000003a     usblib_coff.lib : usbmode.obj (.text:_USB0DualModeIntHandler)
                  00084913    0000003a                     : usbmode.obj (.text:_USBOTGSetMode)
                  0008494d    00000039                     : usbdbulk.obj (.text:_ProcessDataToHost)
                  00084986    00000039     driverlib_coff.lib : usb.obj (.text:_USBIntStatusControl)
                  000849bf    00000038                        : gpio.obj (.text:_GPIO_setMasterCore)
                  000849f7    00000038                        : gpio.obj (.text:_GPIO_setQualificationMode)
                  00084a2f    00000037                        : gpio.obj (.text:_GPIO_setPinConfig)
                  00084a66    00000035                        : gpio.obj (.text:_GPIO_setAnalogMode)
                  00084a9b    00000035     usblib_coff.lib : usbdbulk.obj (.text:_HandleEndpoints)
                  00084ad0    00000034                     : usbdbulk.obj (.text:_HandleDevice)
                  00084b04    00000034     driverlib_coff.lib : interrupt.obj (.text:_Interrupt_enable)
                  00084b38    00000034     usblib_coff.lib : usbbuffer.obj (.text:_USBBufferInit)
                  00084b6c    00000031     driverlib_coff.lib : gpio.obj (.text:_GPIO_setDirectionMode)
                  00084b9d    00000031     usblib_coff.lib : usbdcdesc.obj (.text:_NextConfigDescGet)
                  00084bce    00000031                     : usbdcdesc.obj (.text:_USBDCDConfigGetInterfaceEndpoint)
                  00084bff    00000031                     : usbdenum.obj (.text:_USBDeviceEnumResetHandler)
                  00084c30    00000030                     : usbtick.obj (.text:_InternalUSBRegisterTickHandler)
                  00084c60    0000002f     driverlib_coff.lib : sysctl.obj (.text:_SysCtl_selectOscSourceAuxPLL)
                  00084c8f    0000002e     usblib_coff.lib : usbdcdesc.obj (.text:_ConfigAlternateInterfaceGet)
                  00084cbd    0000002e                     : usbdenum.obj (.text:_USBDSetAddress)
                  00084ceb    0000002c                     : usbdbulk.obj (.text:_HandleConfigChange)
                  00084d17    0000002c                     : usbdenum.obj (.text:_SysCtl_resetPeripheral)
                  00084d43    0000002c                     : usbringbuf.obj (.text:_USBRingBufInit)
                  00084d6f    0000002b                     : usbdma.obj (.text:_DMAUSBIntHandler)
                  00084d9a    0000002b                     : usbtick.obj (.text:_InternalUSBStartOfFrameTick)
                  00084dc5    0000002b                     : usbdesc.obj (.text:_USBDescGet)
                  00084df0    0000002a                     : usbdbulk.obj (.text:_BulkTickHandler)
                  00084e1a    00000029     rts2800_fpu32.lib : exit.c.obj (.text)
                  00084e43    00000028     driverlib_coff.lib : flash.obj (.text:_Flash_setBankPowerUpDelay)
                  00084e6b    00000028     usblib_coff.lib : usbbuffer.obj (.text:_USBBufferInfoGet)
                  00084e93    00000028                     : usbdbulk.obj (.text:_USBDBulkRxPacketAvailable)
                  00084ebb    00000028                     : usbdenum.obj (.text:_USBDeviceResumeTickHandler)
                  00084ee3    00000026                     : usbdesc.obj (.text:_USBDescGetNum)
                  00084f09    00000025                     : usbtick.obj (.text:_InternalUSBTickInit)
                  00084f2e    00000025                     : usbdcdesc.obj (.text:_USBDCDConfigDescGetNum)
                  00084f53    00000024                     : usbringbuf.obj (.text:_USBRingBufContigFree)
                  00084f77    00000024     rts2800_fpu32.lib : cpy_tbl.c.obj (.text)
                  00084f9b    00000023     usblib_coff.lib : usbhostenum.obj (.text:_InternalUSBHCDSendEvent)
                  00084fbe    00000021     driverlib_coff.lib : usb.obj (.text:_USBHostResume)
                  00084fdf    00000021                        : usb.obj (.text:_USBOTGSessionRequest)
                  00085000    00000020                        : interrupt.obj (.text:_Interrupt_initVectorTable)
                  00085020    00000020     usblib_coff.lib : usbdenum.obj (.text:_USBDCDDeviceInfoInit)
                  00085040    00000020                     : usbringbuf.obj (.text:_USBRingBufAdvanceRead)
                  00085060    0000001f                     : usbbuffer.obj (.text:_HandleRequestBuffer)
                  0008507f    0000001f     driverlib_coff.lib : sci.obj (.text:_SCI_isBaseValid)
                  0008509e    0000001f     usblib_coff.lib : usbmode.obj (.text:_USBOTGRemovePower)
                  000850bd    0000001f                     : usbmode.obj (.text:_USBStackModeSet)
                  000850dc    0000001d     rts2800_fpu32.lib : memcpy.c.obj (.text)
                  000850f9    0000001c     usblib_coff.lib : usbdconfig.obj (.text:_GetEndpointFIFOSize)
                  00085115    0000001c     driverlib_coff.lib : usb.obj (.text:_USBIntEnableEndpoint)
                  00085131    0000001b     rts2800_fpu32.lib : fd_toul28.asm.obj (.text)
                  0008514c    0000001a     driverlib_coff.lib : sysctl.obj (.text:_SysCtl_getLowSpeedClock)
                  00085166    0000001a     usblib_coff.lib : usbbuffer.obj (.text:_USBBufferDataWritten)
                  00085180    0000001a                     : usbdenum.obj (.text:_USBDCDStallEP0)
                  0008519a    0000001a                     : usbringbuf.obj (.text:_USBRingBufUsed)
                  000851b4    0000001a                     : usbringbuf.obj (.text:_UpdateIndexAtomic)
                  000851ce    00000019     driverlib_coff.lib : sci.obj (.text:_SCI_disableModule)
                  000851e7    00000019     usblib_coff.lib : usbdbulk.obj (.text:_USBDBulkTxPacketAvailable)
                  00085200    00000019                     : usbdcdesc.obj (.text:_USBDCDConfigDescGetSize)
                  00085219    00000019                     : usbdcdesc.obj (.text:_USBDCDConfigGetInterface)
                  00085232    00000019                     : usbringbuf.obj (.text:_USBRingBufContigUsed)
                  0008524b    00000019     rts2800_fpu32.lib : args_main.c.obj (.text)
                  00085264    00000018     usblib_coff.lib : usbdbulk.obj (.text:_HandleResume)
                  0008527c    00000018                     : usbdbulk.obj (.text:_HandleSuspend)
                  00085294    00000018     driverlib_coff.lib : usb.obj (.text:_USBIntStatusEndpoint)
                  000852ac    00000017     usblib_coff.lib : usbdenum.obj (.text:_SysCtl_enablePeripheral)
                  000852c3    00000017     driverlib_coff.lib : usb.obj (.text:_USBDevDisconnect)
                  000852da    00000017                        : usb.obj (.text:_USBDevMode)
                  000852f1    00000017                        : usb.obj (.text:_USBHostPwrDisable)
                  00085308    00000017                        : usb.obj (.text:_USBHostPwrEnable)
                  0008531f    00000017                        : usb.obj (.text:_USBModeGet)
                  00085336    00000017                        : usb.obj (.text:_USBOTGMode)
                  0008534d    00000016                        : usb.obj (.text:_USBDevConnect)
                  00085363    00000016     usblib_coff.lib : usbringbuf.obj (.text:_USBRingBufFlush)
                  00085379    00000016     rts2800_fpu32.lib : ul_tofd28.asm.obj (.text)
                  0008538f    00000015     usblib_coff.lib : usbbuffer.obj (.text:_HandleDataRemaining)
                  000853a4    00000015                     : usbringbuf.obj (.text:_USBRingBufFree)
                  000853b9    00000014     driverlib_coff.lib : sci.obj (.text:_SCI_enableModule)
                  000853cd    00000014     usblib_coff.lib : usbdenum.obj (.text:_SysCtl_deviceCal)
                  000853e1    00000014     driverlib_coff.lib : usb.obj (.text:_USBHostSuspend)
                  000853f5    00000013     usblib_coff.lib : usbbuffer.obj (.text:_USBBufferFlush)
                  00085408    00000013                     : usbbuffer.obj (.text:_USBBufferSpaceAvailable)
                  0008541b    00000013     driverlib_coff.lib : usb.obj (.text:_USBDevAddrSet)
                  0008542e    00000012     usblib_coff.lib : usbdbulk.obj (.text:_SetDeferredOpFlag)
                  00085440    00000012                     : usbdhandler.obj (.text:_USB0DeviceIntHandler)
                  00085452    00000012                     : usbhostenum.obj (.text:_USB0HostIntHandler)
                  00085464    00000010     driverlib_coff.lib : flash.obj (.text:_Flash_isCtrlBaseValid)
                  00085474    00000010                        : flash.obj (.text:_Flash_isECCBaseValid)
                  00085484    00000010     usblib_coff.lib : usbdenum.obj (.text:_USBDSetDescriptor)
                  00085494    00000010                     : usbdenum.obj (.text:_USBDSyncFrame)
                  000854a4    0000000f                     : usbbuffer.obj (.text:_HandleTxComplete)
                  000854b3    0000000e     driverlib_coff.lib : gpio.obj (.text:_GPIO_isPinValid)
                  000854c1    0000000e                        : interrupt.obj (.text:_Interrupt_defaultHandler)
                  000854cf    0000000e     rts2800_fpu32.lib : fd_sub28.asm.obj (.text)
                  000854dd    0000000d     driverlib_coff.lib : interrupt.obj (.text:_Interrupt_disableMaster)
                  000854ea    0000000d     usblib_coff.lib : usbringbuf.obj (.text:_Interrupt_disableMaster)
                  000854f7    0000000d     driverlib_coff.lib : interrupt.obj (.text:_Interrupt_enableMaster)
                  00085504    0000000d     usblib_coff.lib : usbringbuf.obj (.text:_Interrupt_enableMaster)
                  00085511    0000000c                     : usbdma.obj (.text:_DMAUSBIntStatusClear)
                  0008551d    0000000b     driverlib_coff.lib : sysctl.obj (.text:_SysCtl_isMCDClockFailureDetected)
                  00085528    0000000b     usblib_coff.lib : usbhostenum.obj (.text:_USBHCDPowerAutomatic)
                  00085533    00000009     driverlib_coff.lib : sysctl.obj (.text:_SysCtl_serviceWatchdog)
                  0008553c    00000009     rts2800_fpu32.lib : _lock.c.obj (.text)
                  00085545    00000007     usblib_coff.lib : usbdma.obj (.text:_uDMAUSBChannelAllocate)
                  0008554c    00000007                     : usbdma.obj (.text:_uDMAUSBChannelStatus)
                  00085553    00000007                     : usbdma.obj (.text:_uDMAUSBTransfer)
                  0008555a    00000005                     : usbdma.obj (.text:_DMAUSBStatus)
                  0008555f    00000005                     : usbdma.obj (.text:_uDMAUSBArbSizeSet)
                  00085564    00000005                     : usbdma.obj (.text:_uDMAUSBChannelDisable)
                  00085569    00000005                     : usbdma.obj (.text:_uDMAUSBChannelEnable)
                  0008556e    00000005                     : usbdma.obj (.text:_uDMAUSBChannelIntDisable)
                  00085573    00000005                     : usbdma.obj (.text:_uDMAUSBChannelIntEnable)
                  00085578    00000005                     : usbdma.obj (.text:_uDMAUSBChannelRelease)
                  0008557d    00000005                     : usbdma.obj (.text:_uDMAUSBIntStatus)
                  00085582    00000005                     : usbdma.obj (.text:_uDMAUSBUnitSizeSet)
                  00085587    00000002     driverlib_coff.lib : interrupt.obj (.text:_Interrupt_illegalOperationHandler)
                  00085589    00000002                        : interrupt.obj (.text:_Interrupt_nmiHandler)
                  0008558b    00000002     rts2800_fpu32.lib : pre_init.c.obj (.text)
                  0008558d    00000001                       : startup.c.obj (.text)

.econst    0    00090000    00000a14     
                  00090000    000000ea     usb_ex4_dev_bulk.obj (.econst:.string)
                  000900ea    000000bf     driverlib_coff.lib : flash.obj (.econst:.string)
                  000901a9    00000001     --HOLE-- [fill = 0]
                  000901aa    000000bc                        : gpio.obj (.econst:.string)
                  00090266    000000bb                        : sci.obj (.econst:.string)
                  00090321    00000001     --HOLE-- [fill = 0]
                  00090322    0000007b     usblib_coff.lib : usbdconfig.obj (.econst:.string)
                  0009039d    00000001     --HOLE-- [fill = 0]
                  0009039e    0000007a                     : usbhostenum.obj (.econst:.string)
                  00090418    00000079                     : usbdbulk.obj (.econst:.string)
                  00090491    00000001     --HOLE-- [fill = 0]
                  00090492    00000079                     : usbdenum.obj (.econst:.string)
                  0009050b    00000001     --HOLE-- [fill = 0]
                  0009050c    00000074                     : usbringbuf.obj (.econst:.string)
                  00090580    00000073                     : usbbuffer.obj (.econst:.string)
                  000905f3    00000001     --HOLE-- [fill = 0]
                  000905f4    00000071                     : usbmode.obj (.econst:.string)
                  00090665    00000001     --HOLE-- [fill = 0]
                  00090666    00000070                     : usbdma.obj (.econst:.string)
                  000906d6    0000006c     scistdio.obj (.econst:.string)
                  00090742    00000063     driverlib_coff.lib : interrupt.obj (.econst:.string)
                  000907a5    00000001     --HOLE-- [fill = 0]
                  000907a6    00000060                        : sysctl.obj (.econst:.string)
                  00090806    0000005d                        : usb.obj (.econst:.string)
                  00090863    00000001     --HOLE-- [fill = 0]
                  00090864    00000048     usb_hal.obj (.econst:.string)
                  000908ac    00000030     usb_ex4_dev_bulk_structs.obj (.econst:_g_pui8ConfigString)
                  000908dc    00000028     usb_ex4_dev_bulk_structs.obj (.econst:_g_pui8DataInterfaceString)
                  00090904    00000028     usb_ex4_dev_bulk_structs.obj (.econst:_g_pui8ProductString)
                  0009092c    00000026     ustdlib.obj (.econst:.string)
                  00090952    00000024     usb_ex4_dev_bulk_structs.obj (.econst:_g_pui8ManufacturerString)
                  00090976    0000001a     usblib_coff.lib : usbdenum.obj (.econst:_g_psUSBDStdRequests)
                  00090990    00000018                     : usbdbulk.obj (.econst:_g_sBulkHandlers)
                  000909a8    00000017                     : usbdbulk.obj (.econst:_g_pui8BulkInterface)
                  000909bf    00000001     --HOLE-- [fill = 0]
                  000909c0    00000013     device.obj (.econst:.string)
                  000909d3    00000012     usb_ex4_dev_bulk_structs.obj (.econst:_g_pui8SerialNumberString)
                  000909e5    00000001     --HOLE-- [fill = 0]
                  000909e6    0000000c     usb_ex4_dev_bulk_structs.obj (.econst:_g_ppui8StringDescriptors)
                  000909f2    0000000c     usb_hal.obj (.econst)
                  000909fe    00000004     usb_ex4_dev_bulk_structs.obj (.econst:_g_pui8LangDescriptor)
                  00090a02    00000004     usblib_coff.lib : usbdbulk.obj (.econst:_g_sBulkConfigHeader)
                  00090a06    00000004                     : usbdbulk.obj (.econst:_g_sBulkConfigSection)
                  00090a0a    00000004                     : usbdbulk.obj (.econst:_g_sBulkInterfaceSection)
                  00090a0e    00000002                     : usbdbulk.obj (.econst:_g_ppBulkConfigDescriptors)
                  00090a10    00000002     scistdio.obj (.econst)
                  00090a12    00000002     ustdlib.obj (.econst)

.ebss      1    0000a800    000007b0     UNINITIALIZED
                  0000a800    0000038e     usblib_coff.lib : usbhostenum.obj (.ebss)
                  0000ab8e    00000032                     : usbdenum.obj (.ebss:_g_psDCDInst)
                  0000abc0    00000100     usb_ex4_dev_bulk_structs.obj (.ebss:_g_pui8USBRxBuffer)
                  0000acc0    00000100     usb_ex4_dev_bulk_structs.obj (.ebss:_g_pui8USBTxBuffer)
                  0000adc0    0000008c     usblib_coff.lib : usbdma.obj (.ebss:_g_psUSBDMAInst)
                  0000ae4c    00000012                     : usbdbulk.obj (.ebss:_g_pui8BulkDeviceDescriptor)
                  0000ae5e    0000000c                     : usbtick.obj (.ebss:_g_pfnTickHandlers)
                  0000ae6a    0000000c                     : usbhostenum.obj (.ebss:_g_pi32USBHActiveDriver)
                  0000ae76    0000000a                     : usbmode.obj (.ebss)
                  0000ae80    00000064     usb_ex4_dev_bulk_structs.obj (.ebss)
                  0000aee4    0000000c     usblib_coff.lib : usbhostenum.obj (.ebss:_g_ppvDriverInstance)
                  0000aef0    0000000c                     : usbtick.obj (.ebss:_g_pvTickInstance)
                  0000aefc    00000004                     : usbdbulk.obj (.ebss:_g_psBulkSections)
                  0000af00    00000040                     : usbdenum.obj (.ebss:_g_pui8DataBufferIn)
                  0000af40    0000003e                     : usbhhub.obj (.ebss)
                  0000af7e    00000002     rts2800_fpu32.lib : _lock.c.obj (.ebss:__lock)
                  0000af80    0000000c     usb_ex4_dev_bulk.obj (.ebss)
                  0000af8c    00000009     usblib_coff.lib : usbdbulk.obj (.ebss:_g_pui8BulkDescriptor)
                  0000af95    00000001     ustdlib.obj (.ebss)
                  0000af96    00000006     device.obj (.ebss)
                  0000af9c    00000006     rts2800_fpu32.lib : exit.c.obj (.ebss)
                  0000afa2    00000006     usblib_coff.lib : usbtick.obj (.ebss)
                  0000afa8    00000002     rts2800_fpu32.lib : _lock.c.obj (.ebss:__unlock)
                  0000afaa    00000002     usblib_coff.lib : usbdenum.obj (.ebss:_g_ppsDevInfo)
                  0000afac    00000002     scistdio.obj (.ebss)
                  0000afae    00000002     usblib_coff.lib : usbdenum.obj (.ebss)

MODULE SUMMARY

       Module                         code    initialized data   uninitialized data
       ------                         ----    ----------------   ------------------
    .\
       usb_ex4_dev_bulk_structs.obj   0       255                612               
       usb_ex4_dev_bulk.obj           525     258                12                
       scistdio.obj                   609     115                2                 
       usb_hal.obj                    401     84                 0                 
       ustdlib.obj                    0       44                 1                 
    +--+------------------------------+-------+------------------+--------------------+
       Total:                         1535    756                627               
                                                                                   
    .\device\
       device.obj                     590     34                 6                 
       F2837xD_CodeStartBranch.obj    2       0                  0                 
    +--+------------------------------+-------+------------------+--------------------+
       Total:                         592     34                 6                 
                                                                                   
    C:\ti\c2000\C2000Ware_3_02_00_00\driverlib\f2837xd\driverlib\ccs\Debug\driverlib_coff.lib
       usb.obj                        1772    93                 0                 
       sysctl.obj                     1218    96                 0                 
       flash.obj                      670     191                0                 
       gpio.obj                       365     188                0                 
       interrupt.obj                  397     99                 0                 
       sci.obj                        138     187                0                 
    +--+------------------------------+-------+------------------+--------------------+
       Total:                         4560    854                0                 
                                                                                   
    C:\ti\c2000\C2000Ware_3_02_00_00\libraries\communications\usb\f2837xd\lib\usblib_coff.lib
       usbdenum.obj                   2362    152                118               
       usbhostenum.obj                950     192                934               
       usbdbulk.obj                   911     222                31                
       usbdconfig.obj                 621     123                0                 
       usbbuffer.obj                  602     115                0                 
       usbringbuf.obj                 408     116                0                 
       usbdma.obj                     223     112                140               
       usbmode.obj                    305     126                10                
       usbdcdesc.obj                  299     0                  0                 
       usbtick.obj                    128     14                 30                
       usbdesc.obj                    81      0                  0                 
       usbhhub.obj                    0       0                  62                
       usbdhandler.obj                18      0                  0                 
    +--+------------------------------+-------+------------------+--------------------+
       Total:                         6908    1172               1325              
                                                                                   
    C:\ti\tools\lib\rts2800_fpu32.lib
       fd_add28.asm.obj               156     0                  0                 
       fd_div28.asm.obj               139     0                  0                 
       fs_div28.asm.obj               136     0                  0                 
       boot28.asm.obj                 86      0                  0                 
       exit.c.obj                     41      14                 6                 
       cpy_tbl.c.obj                  36      0                  0                 
       memcpy.c.obj                   29      0                  0                 
       fd_toul28.asm.obj              27      0                  0                 
       args_main.c.obj                25      0                  0                 
       _lock.c.obj                    9       10                 4                 
       ul_tofd28.asm.obj              22      0                  0                 
       fd_sub28.asm.obj               14      0                  0                 
       pre_init.c.obj                 2       0                  0                 
       startup.c.obj                  1       0                  0                 
    +--+------------------------------+-------+------------------+--------------------+
       Total:                         723     24                 10                
                                                                                   
       Stack:                         0       0                  1016              
    +--+------------------------------+-------+------------------+--------------------+
       Grand Total:                   14318   2840               2984              


GLOBAL DATA SYMBOLS: SORTED BY DATA PAGE

address     data page           name
--------    ----------------    ----
00000400      10 (00000400)     __stack

0000ab8e     2ae (0000ab80)     _g_psDCDInst

0000abc0     2af (0000abc0)     _g_pui8USBRxBuffer

0000acc0     2b3 (0000acc0)     _g_pui8USBTxBuffer

0000ae4c     2b9 (0000ae40)     _g_pui8BulkDeviceDescriptor
0000ae5e     2b9 (0000ae40)     _g_pfnTickHandlers
0000ae76     2b9 (0000ae40)     _g_iUSBMode
0000ae77     2b9 (0000ae40)     _g_eOTGModeState
0000ae7a     2b9 (0000ae40)     _g_ui32PollRate
0000ae7c     2b9 (0000ae40)     _g_ui32WaitTicks

0000ae80     2ba (0000ae80)     _g_sRxBuffer
0000ae9c     2ba (0000ae80)     _g_sTxBuffer

0000aec0     2bb (0000aec0)     _g_sBulkDevice
0000aef0     2bb (0000aec0)     _g_pvTickInstance
0000aefc     2bb (0000aec0)     _g_psBulkSections

0000af7e     2bd (0000af40)     __lock

0000af80     2be (0000af80)     _g_eCurrentUSBMode
0000af82     2be (0000af80)     _g_ui32TxCount
0000af84     2be (0000af80)     _g_ui32RxCount
0000af86     2be (0000af80)     _g_ui32SCIRxErrors
0000af88     2be (0000af80)     _g_ui32Flags
0000af8a     2be (0000af80)     _g_pcStatus
0000af8c     2be (0000af80)     _g_pui8BulkDescriptor
0000af96     2be (0000af80)     _Example_Result
0000af98     2be (0000af80)     _Example_PassCount
0000af9a     2be (0000af80)     _Example_Fail
0000af9c     2be (0000af80)     ___TI_enable_exit_profile_output
0000af9e     2be (0000af80)     ___TI_cleanup_ptr
0000afa0     2be (0000af80)     ___TI_dtors_ptr
0000afa2     2be (0000af80)     _g_bUSBTimerInitialized
0000afa4     2be (0000af80)     _g_ui32CurrentUSBTick
0000afa6     2be (0000af80)     _g_ui32USBSOFCount
0000afa8     2be (0000af80)     __unlock
0000afaa     2be (0000af80)     _g_ppsDevInfo

000908ac    2422 (00090880)     _g_pui8ConfigString

000908dc    2423 (000908c0)     _g_pui8DataInterfaceString

00090904    2424 (00090900)     _g_pui8ProductString

00090952    2425 (00090940)     _g_pui8ManufacturerString

00090990    2426 (00090980)     _g_sBulkHandlers
000909a8    2426 (00090980)     _g_pui8BulkInterface

000909d3    2427 (000909c0)     _g_pui8SerialNumberString
000909e6    2427 (000909c0)     _g_ppui8StringDescriptors
000909fe    2427 (000909c0)     _g_pui8LangDescriptor

00090a02    2428 (00090a00)     _g_sBulkConfigHeader
00090a06    2428 (00090a00)     _g_sBulkConfigSection
00090a0a    2428 (00090a00)     _g_sBulkInterfaceSection
00090a0e    2428 (00090a00)     _g_ppBulkConfigDescriptors


GLOBAL SYMBOLS: SORTED ALPHABETICALLY BY Name 

page  address   name                                      
----  -------   ----                                      
abs   ffffffff  .text                                     
0     00084e1a  C$$EXIT                                   
0     000834e0  FD$$ADD                                   
0     00083746  FD$$DIV                                   
0     000854cf  FD$$SUB                                   
0     00085131  FD$$TOUL                                  
0     0008396c  FS$$DIV                                   
0     00085379  UL$$TOFD                                  
0     000831a9  _CPUTimerInit                             
0     00082ba0  _ConfigureSCI                             
0     000827e2  _Device_configureTMXAnalogTrim            
0     00082686  _Device_enableAllPeripherals              
0     000827cc  _Device_enableUnbondedGPIOPullups         
0     000827a9  _Device_enableUnbondedGPIOPullupsFor100Pin
0     00082792  _Device_enableUnbondedGPIOPullupsFor176Pin
0     00082631  _Device_init                              
0     00082771  _Device_initGPIO                          
1     0000af9a  _Example_Fail                             
1     0000af98  _Example_PassCount                        
1     0000af96  _Example_Result                           
0     00082824  _Example_done                             
0     0008281f  _Example_setResultFail                    
0     0008281a  _Example_setResultPass                    
0     00008000  _Flash_initModule                         
0     00084a66  _GPIO_setAnalogMode                       
0     00084b6c  _GPIO_setDirectionMode                    
0     000849bf  _GPIO_setMasterCore                       
0     00084317  _GPIO_setPadConfig                        
0     00084a2f  _GPIO_setPinConfig                        
0     000849f7  _GPIO_setQualificationMode                
0     00084f9b  _InternalUSBHCDSendEvent                  
0     00084c30  _InternalUSBRegisterTickHandler           
0     00084d9a  _InternalUSBStartOfFrameTick              
0     00084f09  _InternalUSBTickInit                      
0     000844f3  _Interrupt_disable                        
0     00084b04  _Interrupt_enable                         
0     000847eb  _Interrupt_initModule                     
0     00085000  _Interrupt_initVectorTable                
0     00082bde  _ModeCallback                             
0     0008612f  _RamfuncsLoadEnd                          
abs   0000012f  _RamfuncsLoadSize                         
0     00086000  _RamfuncsLoadStart                        
0     0000812f  _RamfuncsRunEnd                           
abs   0000012f  _RamfuncsRunSize                          
0     00008000  _RamfuncsRunStart                         
0     00082b6a  _RxHandler                                
0     000823ca  _SCIStdioConfig                           
0     000847ad  _SCI_setConfig                            
0     000825cc  _SCIprintf                                
0     0008240b  _SCIvprintf                               
0     000823da  _SCIwrite                                 
0     0000812b  _SysCtl_delay                             
0     00084369  _SysCtl_getClock                          
0     00083dec  _SysCtl_getDeviceParametric               
0     0008514c  _SysCtl_getLowSpeedClock                  
0     00083f20  _SysCtl_selectOscSource                   
0     00084c60  _SysCtl_selectOscSourceAuxPLL             
0     00082dfe  _SysCtl_setAuxClock                       
0     00082825  _SysCtl_setClock                          
0     00082b54  _TxHandler                                
0     00085440  _USB0DeviceIntHandler                     
0     000848d9  _USB0DualModeIntHandler                   
0     00085452  _USB0HostIntHandler                       
0     00083a79  _USB0OTGModeIntHandler                    
0     00085166  _USBBufferDataWritten                     
0     000846a5  _USBBufferEventCallback                   
0     000853f5  _USBBufferFlush                           
0     00084e6b  _USBBufferInfoGet                         
0     00084b38  _USBBufferInit                            
0     00085408  _USBBufferSpaceAvailable                  
0     0008357c  _USBDBulkCompositeInit                    
0     0008405c  _USBDBulkInit                             
0     00083f7e  _USBDBulkPacketRead                       
0     00084457  _USBDBulkPacketWrite                      
0     00084e93  _USBDBulkRxPacketAvailable                
0     000851e7  _USBDBulkTxPacketAvailable                
0     00084661  _USBDCDConfigDescGet                      
0     00084f2e  _USBDCDConfigDescGetNum                   
0     00085200  _USBDCDConfigDescGetSize                  
0     00085219  _USBDCDConfigGetInterface                 
0     00084bce  _USBDCDConfigGetInterfaceEndpoint         
0     00085020  _USBDCDDeviceInfoInit                     
0     00083433  _USBDCDInit                               
0     00085180  _USBDCDStallEP0                           
0     000831c4  _USBDelay                                 
0     00084dc5  _USBDescGet                               
0     00084ee3  _USBDescGetNum                            
0     0008541b  _USBDevAddrSet                            
0     0008534d  _USBDevConnect                            
0     000852c3  _USBDevDisconnect                         
0     0008385b  _USBDevEndpointConfigSet                  
0     00084588  _USBDevEndpointDataAck                    
0     000840b7  _USBDevEndpointStall                      
0     00083b69  _USBDevEndpointStallClear                 
0     00083d19  _USBDevEndpointStatusClear                
0     000852da  _USBDevMode                               
0     00082c51  _USBDeviceConfig                          
0     00083d83  _USBDeviceConfigAlternate                 
0     000831f7  _USBDeviceEnumHandler                     
0     00084bff  _USBDeviceEnumResetHandler                
0     00083617  _USBDeviceIntHandlerInternal              
0     00084ebb  _USBDeviceResumeTickHandler               
0     0008461a  _USBEndpointDataAvail                     
0     00083cae  _USBEndpointDataGet                       
0     00084270  _USBEndpointDataPut                       
0     00084112  _USBEndpointDataSend                      
0     0008476e  _USBEndpointStatus                        
0     00083e54  _USBFIFOConfigSet                         
0     00083198  _USBGPIOEnable                            
0     00085528  _USBHCDPowerAutomatic                     
0     000846e8  _USBHostEndpointDataAck                   
0     000843ba  _USBHostEndpointStatusClear               
0     00082000  _USBHostIntHandlerInternal                
0     000852f1  _USBHostPwrDisable                        
0     00085308  _USBHostPwrEnable                         
0     00084fbe  _USBHostResume                            
0     000853e1  _USBHostSuspend                           
0     0008489e  _USBIntEnableControl                      
0     00085115  _USBIntEnableEndpoint                     
0     000841c3  _USBIntStatus                             
0     00084986  _USBIntStatusControl                      
0     00085294  _USBIntStatusEndpoint                     
0     00083eba  _USBLibDMAInit                            
0     0008531f  _USBModeGet                               
0     00085336  _USBOTGMode                               
0     00084fdf  _USBOTGSessionRequest                     
0     00085040  _USBRingBufAdvanceRead                    
0     0008472b  _USBRingBufAdvanceWrite                   
0     00084f53  _USBRingBufContigFree                     
0     00085232  _USBRingBufContigUsed                     
0     00085363  _USBRingBufFlush                          
0     000853a4  _USBRingBufFree                           
0     00084d43  _USBRingBufInit                           
0     0008519a  _USBRingBufUsed                           
0     000842c4  _USBRingBufWrite                          
0     000850bd  _USBStackModeSet                          
1     000007f8  __STACK_END                               
abs   000003f8  __STACK_SIZE                              
1     0000af9e  ___TI_cleanup_ptr                         
1     0000afa0  ___TI_dtors_ptr                           
1     0000af9c  ___TI_enable_exit_profile_output          
abs   ffffffff  ___TI_pprof_out_hndl                      
abs   ffffffff  ___TI_prof_data_size                      
abs   ffffffff  ___TI_prof_data_start                     
abs   ffffffff  ___binit__                                
abs   ffffffff  ___c_args__                               
0     00088000  ___cinit__                                
0     00082813  ___error__                                
abs   ffffffff  ___etext__                                
abs   ffffffff  ___pinit__                                
abs   ffffffff  ___text__                                 
0     0008524b  __args_main                               
1     0000af7e  __lock                                    
0     00085544  __nop                                     
0     00085540  __register_lock                           
0     0008553c  __register_unlock                         
1     00000400  __stack                                   
0     0008558d  __system_post_cinit                       
0     0008558b  __system_pre_init                         
1     0000afa8  __unlock                                  
0     00084e1a  _abort                                    
0     0008421a  _c_int00                                  
0     00084f77  _copy_in                                  
0     00084e1c  _exit                                     
0     000832c1  _f28x_USB0DeviceIntHandler                
0     00083323  _f28x_USB0DualModeIntHandler              
0     000832f2  _f28x_USB0HostIntHandler                  
0     00083354  _f28x_USB0OTGModeIntHandler               
1     0000afa2  _g_bUSBTimerInitialized                   
1     0000af80  _g_eCurrentUSBMode                        
1     0000ae77  _g_eOTGModeState                          
1     0000ae76  _g_iUSBMode                               
1     0000af8a  _g_pcStatus                               
1     0000ae5e  _g_pfnTickHandlers                        
0     00090a0e  _g_ppBulkConfigDescriptors                
1     0000afaa  _g_ppsDevInfo                             
0     000909e6  _g_ppui8StringDescriptors                 
1     0000aefc  _g_psBulkSections                         
1     0000ab8e  _g_psDCDInst                              
1     0000af8c  _g_pui8BulkDescriptor                     
1     0000ae4c  _g_pui8BulkDeviceDescriptor               
0     000909a8  _g_pui8BulkInterface                      
0     000908ac  _g_pui8ConfigString                       
0     000908dc  _g_pui8DataInterfaceString                
0     000909fe  _g_pui8LangDescriptor                     
0     00090952  _g_pui8ManufacturerString                 
0     00090904  _g_pui8ProductString                      
0     000909d3  _g_pui8SerialNumberString                 
1     0000abc0  _g_pui8USBRxBuffer                        
1     0000acc0  _g_pui8USBTxBuffer                        
1     0000aef0  _g_pvTickInstance                         
0     00090a02  _g_sBulkConfigHeader                      
0     00090a06  _g_sBulkConfigSection                     
1     0000aec0  _g_sBulkDevice                            
0     00090990  _g_sBulkHandlers                          
0     00090a0a  _g_sBulkInterfaceSection                  
1     0000ae80  _g_sRxBuffer                              
1     0000ae9c  _g_sTxBuffer                              
1     0000afa4  _g_ui32CurrentUSBTick                     
1     0000af88  _g_ui32Flags                              
1     0000ae7a  _g_ui32PollRate                           
1     0000af84  _g_ui32RxCount                            
1     0000af86  _g_ui32SCIRxErrors                        
1     0000af82  _g_ui32TxCount                            
1     0000afa6  _g_ui32USBSOFCount                        
1     0000ae7c  _g_ui32WaitTicks                          
0     00082be7  _main                                     
0     000850dc  _memcpy                                   
abs   ffffffff  binit                                     
0     00088000  cinit                                     
0     00080000  code_start                                
abs   ffffffff  etext                                     
abs   ffffffff  pinit                                     


GLOBAL SYMBOLS: SORTED BY Symbol Address 

page  address   name                                      
----  -------   ----                                      
0     00008000  _Flash_initModule                         
0     00008000  _RamfuncsRunStart                         
0     0000812b  _SysCtl_delay                             
0     0000812f  _RamfuncsRunEnd                           
0     00080000  code_start                                
0     00082000  _USBHostIntHandlerInternal                
0     000823ca  _SCIStdioConfig                           
0     000823da  _SCIwrite                                 
0     0008240b  _SCIvprintf                               
0     000825cc  _SCIprintf                                
0     00082631  _Device_init                              
0     00082686  _Device_enableAllPeripherals              
0     00082771  _Device_initGPIO                          
0     00082792  _Device_enableUnbondedGPIOPullupsFor176Pin
0     000827a9  _Device_enableUnbondedGPIOPullupsFor100Pin
0     000827cc  _Device_enableUnbondedGPIOPullups         
0     000827e2  _Device_configureTMXAnalogTrim            
0     00082813  ___error__                                
0     0008281a  _Example_setResultPass                    
0     0008281f  _Example_setResultFail                    
0     00082824  _Example_done                             
0     00082825  _SysCtl_setClock                          
0     00082b54  _TxHandler                                
0     00082b6a  _RxHandler                                
0     00082ba0  _ConfigureSCI                             
0     00082bde  _ModeCallback                             
0     00082be7  _main                                     
0     00082c51  _USBDeviceConfig                          
0     00082dfe  _SysCtl_setAuxClock                       
0     00083198  _USBGPIOEnable                            
0     000831a9  _CPUTimerInit                             
0     000831c4  _USBDelay                                 
0     000831f7  _USBDeviceEnumHandler                     
0     000832c1  _f28x_USB0DeviceIntHandler                
0     000832f2  _f28x_USB0HostIntHandler                  
0     00083323  _f28x_USB0DualModeIntHandler              
0     00083354  _f28x_USB0OTGModeIntHandler               
0     00083433  _USBDCDInit                               
0     000834e0  FD$$ADD                                   
0     0008357c  _USBDBulkCompositeInit                    
0     00083617  _USBDeviceIntHandlerInternal              
0     00083746  FD$$DIV                                   
0     0008385b  _USBDevEndpointConfigSet                  
0     0008396c  FS$$DIV                                   
0     00083a79  _USB0OTGModeIntHandler                    
0     00083b69  _USBDevEndpointStallClear                 
0     00083cae  _USBEndpointDataGet                       
0     00083d19  _USBDevEndpointStatusClear                
0     00083d83  _USBDeviceConfigAlternate                 
0     00083dec  _SysCtl_getDeviceParametric               
0     00083e54  _USBFIFOConfigSet                         
0     00083eba  _USBLibDMAInit                            
0     00083f20  _SysCtl_selectOscSource                   
0     00083f7e  _USBDBulkPacketRead                       
0     0008405c  _USBDBulkInit                             
0     000840b7  _USBDevEndpointStall                      
0     00084112  _USBEndpointDataSend                      
0     000841c3  _USBIntStatus                             
0     0008421a  _c_int00                                  
0     00084270  _USBEndpointDataPut                       
0     000842c4  _USBRingBufWrite                          
0     00084317  _GPIO_setPadConfig                        
0     00084369  _SysCtl_getClock                          
0     000843ba  _USBHostEndpointStatusClear               
0     00084457  _USBDBulkPacketWrite                      
0     000844f3  _Interrupt_disable                        
0     00084588  _USBDevEndpointDataAck                    
0     0008461a  _USBEndpointDataAvail                     
0     00084661  _USBDCDConfigDescGet                      
0     000846a5  _USBBufferEventCallback                   
0     000846e8  _USBHostEndpointDataAck                   
0     0008472b  _USBRingBufAdvanceWrite                   
0     0008476e  _USBEndpointStatus                        
0     000847ad  _SCI_setConfig                            
0     000847eb  _Interrupt_initModule                     
0     0008489e  _USBIntEnableControl                      
0     000848d9  _USB0DualModeIntHandler                   
0     00084986  _USBIntStatusControl                      
0     000849bf  _GPIO_setMasterCore                       
0     000849f7  _GPIO_setQualificationMode                
0     00084a2f  _GPIO_setPinConfig                        
0     00084a66  _GPIO_setAnalogMode                       
0     00084b04  _Interrupt_enable                         
0     00084b38  _USBBufferInit                            
0     00084b6c  _GPIO_setDirectionMode                    
0     00084bce  _USBDCDConfigGetInterfaceEndpoint         
0     00084bff  _USBDeviceEnumResetHandler                
0     00084c30  _InternalUSBRegisterTickHandler           
0     00084c60  _SysCtl_selectOscSourceAuxPLL             
0     00084d43  _USBRingBufInit                           
0     00084d9a  _InternalUSBStartOfFrameTick              
0     00084dc5  _USBDescGet                               
0     00084e1a  C$$EXIT                                   
0     00084e1a  _abort                                    
0     00084e1c  _exit                                     
0     00084e6b  _USBBufferInfoGet                         
0     00084e93  _USBDBulkRxPacketAvailable                
0     00084ebb  _USBDeviceResumeTickHandler               
0     00084ee3  _USBDescGetNum                            
0     00084f09  _InternalUSBTickInit                      
0     00084f2e  _USBDCDConfigDescGetNum                   
0     00084f53  _USBRingBufContigFree                     
0     00084f77  _copy_in                                  
0     00084f9b  _InternalUSBHCDSendEvent                  
0     00084fbe  _USBHostResume                            
0     00084fdf  _USBOTGSessionRequest                     
0     00085000  _Interrupt_initVectorTable                
0     00085020  _USBDCDDeviceInfoInit                     
0     00085040  _USBRingBufAdvanceRead                    
0     000850bd  _USBStackModeSet                          
0     000850dc  _memcpy                                   
0     00085115  _USBIntEnableEndpoint                     
0     00085131  FD$$TOUL                                  
0     0008514c  _SysCtl_getLowSpeedClock                  
0     00085166  _USBBufferDataWritten                     
0     00085180  _USBDCDStallEP0                           
0     0008519a  _USBRingBufUsed                           
0     000851e7  _USBDBulkTxPacketAvailable                
0     00085200  _USBDCDConfigDescGetSize                  
0     00085219  _USBDCDConfigGetInterface                 
0     00085232  _USBRingBufContigUsed                     
0     0008524b  __args_main                               
0     00085294  _USBIntStatusEndpoint                     
0     000852c3  _USBDevDisconnect                         
0     000852da  _USBDevMode                               
0     000852f1  _USBHostPwrDisable                        
0     00085308  _USBHostPwrEnable                         
0     0008531f  _USBModeGet                               
0     00085336  _USBOTGMode                               
0     0008534d  _USBDevConnect                            
0     00085363  _USBRingBufFlush                          
0     00085379  UL$$TOFD                                  
0     000853a4  _USBRingBufFree                           
0     000853e1  _USBHostSuspend                           
0     000853f5  _USBBufferFlush                           
0     00085408  _USBBufferSpaceAvailable                  
0     0008541b  _USBDevAddrSet                            
0     00085440  _USB0DeviceIntHandler                     
0     00085452  _USB0HostIntHandler                       
0     000854cf  FD$$SUB                                   
0     00085528  _USBHCDPowerAutomatic                     
0     0008553c  __register_unlock                         
0     00085540  __register_lock                           
0     00085544  __nop                                     
0     0008558b  __system_pre_init                         
0     0008558d  __system_post_cinit                       
0     00086000  _RamfuncsLoadStart                        
0     0008612f  _RamfuncsLoadEnd                          
0     00088000  ___cinit__                                
0     00088000  cinit                                     
0     000908ac  _g_pui8ConfigString                       
0     000908dc  _g_pui8DataInterfaceString                
0     00090904  _g_pui8ProductString                      
0     00090952  _g_pui8ManufacturerString                 
0     00090990  _g_sBulkHandlers                          
0     000909a8  _g_pui8BulkInterface                      
0     000909d3  _g_pui8SerialNumberString                 
0     000909e6  _g_ppui8StringDescriptors                 
0     000909fe  _g_pui8LangDescriptor                     
0     00090a02  _g_sBulkConfigHeader                      
0     00090a06  _g_sBulkConfigSection                     
0     00090a0a  _g_sBulkInterfaceSection                  
0     00090a0e  _g_ppBulkConfigDescriptors                
1     00000400  __stack                                   
1     000007f8  __STACK_END                               
1     0000ab8e  _g_psDCDInst                              
1     0000abc0  _g_pui8USBRxBuffer                        
1     0000acc0  _g_pui8USBTxBuffer                        
1     0000ae4c  _g_pui8BulkDeviceDescriptor               
1     0000ae5e  _g_pfnTickHandlers                        
1     0000ae76  _g_iUSBMode                               
1     0000ae77  _g_eOTGModeState                          
1     0000ae7a  _g_ui32PollRate                           
1     0000ae7c  _g_ui32WaitTicks                          
1     0000ae80  _g_sRxBuffer                              
1     0000ae9c  _g_sTxBuffer                              
1     0000aec0  _g_sBulkDevice                            
1     0000aef0  _g_pvTickInstance                         
1     0000aefc  _g_psBulkSections                         
1     0000af7e  __lock                                    
1     0000af80  _g_eCurrentUSBMode                        
1     0000af82  _g_ui32TxCount                            
1     0000af84  _g_ui32RxCount                            
1     0000af86  _g_ui32SCIRxErrors                        
1     0000af88  _g_ui32Flags                              
1     0000af8a  _g_pcStatus                               
1     0000af8c  _g_pui8BulkDescriptor                     
1     0000af96  _Example_Result                           
1     0000af98  _Example_PassCount                        
1     0000af9a  _Example_Fail                             
1     0000af9c  ___TI_enable_exit_profile_output          
1     0000af9e  ___TI_cleanup_ptr                         
1     0000afa0  ___TI_dtors_ptr                           
1     0000afa2  _g_bUSBTimerInitialized                   
1     0000afa4  _g_ui32CurrentUSBTick                     
1     0000afa6  _g_ui32USBSOFCount                        
1     0000afa8  __unlock                                  
1     0000afaa  _g_ppsDevInfo                             
abs   0000012f  _RamfuncsLoadSize                         
abs   0000012f  _RamfuncsRunSize                          
abs   000003f8  __STACK_SIZE                              
abs   ffffffff  .text                                     
abs   ffffffff  ___TI_pprof_out_hndl                      
abs   ffffffff  ___TI_prof_data_size                      
abs   ffffffff  ___TI_prof_data_start                     
abs   ffffffff  ___binit__                                
abs   ffffffff  ___c_args__                               
abs   ffffffff  ___etext__                                
abs   ffffffff  ___pinit__                                
abs   ffffffff  ___text__                                 
abs   ffffffff  binit                                     
abs   ffffffff  etext                                     
abs   ffffffff  pinit                                     

[213 symbols]
